:02000000842951
:080008000000000009000130B6
:10001000A9000130AA000530AB0038280130A90042
:100020000130AA002030AB0038280130A90002308E
:10003000AA00F330AB0038280130A9000830AA002C
:10004000CD30AB0038280130A9004F30AA00013074
:10005000AB0038280230A9008730AA006A30AB0014
:1000600038281030A9002830AA00C830AB00382842
:10007000AB0B3828AA0B3828A90B38280800000039
:10008000000000000000080097010130B52015288D
:1000900097010830A8008030B52015202030692055
:1000A000A80B4E288030B5209701152897010830FD
:1000B000A800C030B520152020306920A80B97017A
:1000C0005C28C030B520970115280230B520970173
:1000D00015288312A60017089719F739803E971D37
:1000E0007228403EB5200E2026080F3086052608CF
:1000F000F0398604000005150000051407200510DE
:1001000007200F308605260EF039860400000514FE
:10011000072005100720970A080005101520051173
:10012000152015200F3086053030860483160F30D9
:10013000060586008312051400000510152005141D
:1001400000000510152005140000051023200F30B5
:100150008605203086040514000005102830B520DF
:100160000830B5200C30B5200630A70023200F3012
:1001700086052708F03986040000051100000514E3
:10018000000005100F308605270EF039860405148F
:10019000000005100800831310088D020318D728EB
:1001A00001308E020318D7288F02031C8317110811
:1001B0008E020318DF2801308F02031C83171208F8
:1001C0008F02031C8317003410088D07031CEB28D3
:1001D0008E0FEB288F0A11088E0703188F0A12085A
:1001E0008F07003407309F00183084002F308000C4
:1001F000840A9F0BF7280F30920042309100403064
:1002000090008313CB20980A3A3018060319DB2993
:10021000831F0229E4200130920086309100A03033
:100220009000CB20990A831F1129E42092012730E6
:10023000910010309000CB209A0A831F1B29E420E4
:1002400003309100E8309000CB209B0A831F2429C3
:10025000E420910164309000CB209C0A831F2C295C
:10026000E4200A309000CB209D0A831F3329E4202C
:100270000D089E079E0A00348316373081008312D2
:10028000851105118F01810196010C089F008515CC
:10029000FA30A00058294C294D294E294F295029C0
:1002A0005129522953295429552956295729582962
:1002B00001089602031D5E290000602903188F0AB9
:1002C0009600000000000000A00B4B296729682958
:1002D00069296A296B296C296D296E296F29702972
:1002E0009F0B4829851101088E009602031C7A296C
:1002F000031D8F0A8D018D030515000005110108EE
:100300000E0603197B2900348501860183161230FD
:10031000850000308600831286152A208D202A2031
:1003200048200030A300F521312048200130A300EF
:10033000F521312048200230A300F521312048204A
:1003400086110830860623200030851864308C0022
:100350003C21F220E2210430970007309F00183042
:10036000840030300006031DBB2920306920840A38
:100370009F0BB129C82900086920840A8518C6295D
:1003800005301F06031DC6292E3069209F0BBB298F
:100390000B309700203069208518D0294D30692016
:1003A000483069207A30692020306920851CA129D5
:1003B00020306920A129970148200330A300F521AE
:1003C0003120A1299701851CED296520463069203F
:1003D000723069207130692008006520563069202C
:1003E0004830692046306920080023088E00031039
:1003F0008E0D8E0D8E0D8E0D8F0197010F080E073D
:1004000089008316081483120E200808003A031985
:0C0410000D2A69208F0A0F1EFE2908002B
:02400E00F13F80
:1042000057344334543438345F344C3443344434B6
:104210002034323478343834203431344C3420343F
:1042200031342D34313430344D3468347A342034E0
:10423000313430342D343934393439344D347A34DE
:1042400052346534763431343334303433343334A7
:10425000303420344E346F3463346F3472347234FB
:104260004F3476346534723466346C346F3477345A
:1042700020342034203420342034203420342E3490
:00000001FF
